:020000040000FA
:100000006030840017208C28A000A00E030EA100F1
:10001000802800088403800008000008A200840AE9
:100020000008A300840A22080A2023080A283B307B
:100030000A2000300A200D208003031D192860309B
:1000400084000800210E8300200E09008312850120
:100050000730990083169F01831208000B178B1736
:100060000800F030A6000800F630A50008009C301B
:10007000A40008003120342037280B118B16823061
:100080008100080029080A200008A807840A08003F
:100090004220F830A80408000008A907840A0800D4
:1000A0000130AA0708005D200130AB070800851663
:1000B00008008512FF30AB0008002B088207572884
:1000C0005928532028080A200008A700840A08009D
:1000D000A70A0319612808005020A9017B30A80055
:1000E000312022282A080A204C203420A60A03198D
:1000F0006C28222848203720A50A031972282228B4
:100100003D206820A40A03197A2822288316640057
:100110008830810083120800262083160F30850066
:10012000831286202E203D203A20FF30A900EC309B
:06013000A8009928080058
:02400E00E43F8D
:00000001FF
